:020000040000FA
:1000000088260020F902000001030000030300001D
:1000100005030000070300000903000000000000C2
:100020000000000000000000000000000B030000C2
:100030000D030000000000000F030000110300008A
:100040001303000013030000A505000013030000C4
:100050001303000013030000130300001303000048
:100060001303000013030000130300001303000038
:1000700013030000A103000013030000130300009A
:100080001303000013030000130300001303000018
:100090001303000013030000130300001303000008
:1000A00013030000130300001303000013030000F8
:1000B0001303000013030000000000000000000014
:1000C00013030000130300001303000013030000D8
:1000D00013030000130300001303000013030000C8
:1000E00013030000130300001303000000000000CE
:1000F00000000000130300000000000013030000D4
:1001000000000000000000000000000000000000EF
:1001100000000000000000000000000000000000DF
:1001200000000000000000000000000000000000CF
:1001300000000000000000000000000000000000BF
:1001400000000000000000000000000000000000AF
:10015000000000000000000000000000000000009F
:10016000000000000000000000000000000000008F
:10017000000000000000000000000000000000007F
:10018000000000000000000000000000000000006F
:10019000000000000000000000000000000000005F
:1001A000000000000000000000000000000000004F
:1001B000000000000000000000000000000000003F
:1001C000000000000000000000000000000000002F
:1001D000000000000000000000000000000000001F
:1001E000000000000000000000000000000000000F
:1001F00000000000000000000000000000000000FF
:10020000DFF80CD000F0BAF8004800475D0A0000A3
:100210008826002030B4044654E8000F0D4644E818
:100220000053002BF8D1156030BC704730B4044641
:1002300054E8000F40EA010544E80053002BF7D1D1
:10024000156030BC704730B4044654E8000F00EA33
:10025000010544E80053002BF7D1156030BC70470E
:1002600030B4044654E8000F80EA010544E8005326
:10027000002BF7D1156030BC704730B4044654E809
:10028000000F00EB010544E80053002BF7D1156087
:1002900030BC704730B4044654E8000FA0EB0105B1
:1002A00044E80053002BF7D1156030BC704770B4A0
:1002B00004464FF0000054E8006F0D68AE4207BFDF
:1002C00044E80023012044E800630E60002B1CBFBB
:1002D0000020F0E770BC704730B4044654E8000FCB
:1002E00088422CBF451A054644E80053002BF5D13F
:1002F000156030BC7047000006488047064800473C
:10030000FEE7FEE7FEE7FEE7FEE7FEE7FEE7FEE7C5
:10031000FEE7FEE7C9030000010200000048704745
:10032000F025000040EA01039B0703D009E008C95B
:10033000121F08C0042AFAD203E011F8013B00F8AA
:10034000013B521EF9D27047D2B201E000F8012BF6
:10035000491EFBD270470022F6E710B513460A4645
:1003600004461946FFF7F0FF204610BD421C10F866
:10037000011B0029FBD1801A70470000064C074D75
:1003800006E0E06840F0010394E807009847103465
:10039000AC42F6D3FFF738FFA4260000C4260000C5
:1003A000064882B00021016000680090044800689F
:1003B0000449C0B2496802B00847000000D10040BB
:1003C00008D500402000002030B54FF080500022BA
:1003D0008300D0F83011C3F80C21C3F81021624B10
:1003E0001A60624B1B68624C2360604B1B1D1B68CC
:1003F000241D23605D4B08331B68241D23605B4B69
:100400000C331B68241D2360584B10331B68241DBC
:100410002360564B14331B68241D2360534B183341
:100420001B68534C20342360504B1C331B68241D25
:1004300023604E4B20331B68241D23604B4B243319
:100440001B68241D2360494B28331B68241D23602F
:10045000464B2C331B68241D2360444B30331B68F0
:10046000434C40342360414B34331B68241D2360CC
:100470003E4B38331B68241D23603C4B3C331B68C8
:10048000241D2360394B40331B68241D2360012445
:10049000082902D1D0F8343113B1082904D006E07C
:1004A000354B3449196005E0D0F8343113B10829CF
:1004B00004D006E0314BFB21196005E0D0F834315F
:1004C00013B1082908D00EE090F858322C48016882
:1004D00063F30301016002E0D0F834311BB929490C
:1004E0004FF40070086028480168C90702D06FF017
:1004F000010101602548016841F470010160BFF30A
:100500004F8FBFF36F8F4FF01021D1F800020028FA
:1005100003DBD1F80402002822DA1D4B1C601D48C1
:100520000468002CFCD01224C1F800420568002D9C
:10053000FCD0C1F8044201680029FCD01A600168AF
:100540000029FCD0BFF34F8F10487C380168124A55
:1005500001F4E06111430160BFF34F8F00BFFDE77D
:100560000F490E48086030BD3805004004040010F3
:1005700020C50040488103008C56004018F500401B
:10058000E40E0040409602400004004088ED00E088
:1005900004E5014000E401400400FA050090D003A6
:1005A000A00000200148006800470000180000205B
:1005B00002E008C8121F08C1002AFAD1704770472C
:1005C000002001E001C1121F002AFBD1704700008A
:1005D00072B601F04DF800BF00F04CFE0028FBD1D0
:1005E000104C0121208801EB00400FA100F0A2FF78
:1005F00010480068C00700D000BE2088022101EB2F
:1006000000400DA100F096FFBFF34F8F0948E4387A
:1006100001680D4A01F4E06111430160BFF34F8F9F
:1006200000BFFDE7C0000020466174616C20657268
:10063000726F7200F0ED00E053797374656D207293
:1006400065736574000000000400FA050EB5002112
:100650000091CDE901106A4644F20100FFF7B8FFAE
:100660000EBD00F003B800F009B8000072B60248F1
:100670000168491C01607047280000200349086890
:10068000401E086000D162B67047000028000020BC
:1006900070B5054608680C46411C04D000F0FEFC0D
:1006A000206800F0CBFC6068411C02D0002100F003
:1006B000B3FC2968A069C1F82405607D227D296802
:1006C0001043C1F86C05D4E900122868C0F814255D
:1006D000C0F80C15207D012814D1A068411C02D05F
:1006E000002100F099FCE068411C04D000F0D6FC29
:1006F000E06800F0A3FCD4E902122868C0F80825DD
:10070000C0F8101570BD70B5054608680C46411C50
:1007100004D000F0CDFC206800F09AFC6068411C19
:1007200002D0002100F081FC2968A069C1F82405ED
:10073000607D217D2A680843C2F86C05D4E9001267
:100740002868C0F80C15C0F81425207D012814D1A4
:10075000A068411C02D0002100F067FCE068411C49
:1007600004D000F0A5FCE06800F072FCD4E90212AD
:100770002868C0F80825C0F8101570BD2DE9F047AD
:100780000546861C90460F464FF001090020FFF7F2
:1007900068FF1B4C20683860D4E90001401AA1684A
:1007A00004F21C47081A0EE00121384600F018FA3E
:1007B00000F006F90146384600F012FAD4E90001CB
:1007C000401AA168081A401C8642EDD8B8F1000F03
:1007D00003D0052065F3891002E0062065F39F50E1
:1007E000A2682168114004EB8101C8602068304490
:1007F00020600020FFF737FF4846BDE8F087000083
:100800006402002030B482680468531C8360A154E1
:10081000D0E901128A4202D330BC00F0C0BA30BC29
:1008200070470000034803C8814201D1012070478E
:10083000002070476402002010B50021024800F03B
:10084000DAF980F3100010BD800600202DE9FC5F6E
:100850000E008346DDE90C47C6F10000984692463B
:10086000814600D40846012503E000BF90FBFAF062
:100870006D1C5045FADAA84500D9454624B1002E32
:1008800001DB780700D5641EB80702D5B8F1000F68
:100890000AD0F80708D13CB1A54205D2202158461C
:1008A000641EFFF7AFFFF6E7002E02DA4E462D2159
:1008B00002E0780703D52B215846FFF7A3FF07F086
:1008C000030002280BD1B8F1000F08D13CB1A542BA
:1008D00005D230215846641EFFF794FFF6E7CDE9B4
:1008E0000047434652463146584601F0BFFDBDE839
:1008F000FC9F000070B50D46044600684FF48871F7
:1009000001F03CF84FF49071206801F037F84FF493
:100910009271206801F032F84FF4A271206801F062
:100920002DF820681249C0F8041320686907000BED
:1009300040B2090E002806DA00F00F0000F1E020B6
:1009400080F8141D03E000F1E02080F80014206816
:100950000121000B40B200F01F02914040098000CD
:1009600000F1E020C0F88012C0F8001170BD000056
:1009700010030200024600201268930702D05307BA
:1009800002D47047500714D502F00300012802D0AA
:1009900002280CD105E0C2F383100B68801C1844B8
:1009A00004E00223086803EB92521044086001201F
:1009B0007047086800EB9253C2F38910401CEEE7C1
:1009C0002DE9FF410026234800F007F92148001FC8
:1009D000074600F002F9204C60680090A56800E02E
:1009E00000986946284004EB80000C30FFF7C2FFF6
:1009F0000028F5D101AA009901EA050304EB83035D
:100A0000491CDB6842F82030401C00910228F2D3D8
:100A1000019800F0030001280BD0022810D10198A2
:100A2000032101EB90500099BDF80A6001EB9000A2
:100A300005E00198BDF80A60C0F3831008440090F7
:100A4000384600F0C7F808B10098606004B030463E
:100A5000BDE8F0817C0600206402002086B04FF4DF
:100A60000041002000F0C0FD08B1FFF7EFFD00F0ED
:100A7000F3FB002000F026F908B1FFF7E7FD1F4D5A
:100A800003241FA1288804EB004000F053FDA84672
:100A90006E46102504A800F00BF99DF810001028F0
:100AA00000D805462946304600F02AF908B1FFF77C
:100AB000CDFDB8F800002E46454604EB004016A1D7
:100AC00000F038FD2888324604EB0040694600F00B
:100AD000DDFC28880FA104EB004000F02BFD00BFD7
:100AE00000F0C8FB0028FBD10F4D64264FF47A4775
:100AF000691C38468847761EFAD1C9E7C000002035
:100B0000524E47206578616D706C65207374617218
:100B10007465642E0000000052616E646F6D205693
:100B20006563746F723A0000202500002DE9F047DC
:100B3000C7880446181D16468946B0FBF7F1B0FB7E
:100B4000F7F207FB12009A193A44D21CB2FBF7F2F3
:100B5000DDF820A001E02468491E0029FBD13D1AE0
:100B60008846B54216D818E0BAF1000F05D0211812
:100B700009EB08002A46091D04E0204409EB08019E
:100B80002A46001DFFF7CEFB00202468761BA844F0
:100B9000B74201D9354600E03D46002EE4D1BDE81C
:100BA000F087000030B5024659B100F049FD002140
:100BB000074C09E004EB810315685B88AB4202D166
:100BC0001160002030BD491C8142F3D3052030BDA7
:100BD000A4000020002100F009B8012100F010B8A5
:100BE00008B56A46FFF749FB009808BD08B56A4694
:100BF000FFF729FB08BD08B56A46FFF70BFB08BDE8
:100C000008B56A46FFF712FB009808BD08B56A46AA
:100C1000FFF740FB009808BD70B504460025284644
:100C2000FFF71FFD21686268086890420ED9401ED8
:100C300008600178A38AE26801FB0325227A216813
:100C4000101AC0B20A79824200D208710020FFF760
:100C50000AFD284670BD70B505460C460020FFF71A
:100C600000FDE868A98A201AB0FBF1F12A68106833
:100C7000431C13600170BDE870400020FFF7F3BC17
:100C800010B530B1017A42680368891AC9B21A6096
:100C900006E00E2010BD03681A68541C1C60117019
:100CA000491EC9B2F7D2006800210171084610BD83
:100CB00010B50446024800F03DFE207010BD000053
:100CC0001C27000070B50B4C217809B1852070BD40
:100CD00000B9094809490088A4F80100601C00F027
:100CE0008DFE0500F3D100F0B7FE012020702846EC
:100CF00070BD00000000002026250000DD19000066
:100D00000A4610B50146044800F0F7FD044600F01D
:100D1000A3FE204610BD00001C270000F0B50546CC
:100D20000478154889B0164640F82420124A08690C
:100D30000832A2F10C0742F82400487F38552022DF
:100D40006846FFF7EFFA04942878385C48B10EB192
:100D50000A4A00E000226946281D00F0CDFF09B0D4
:100D6000F0BD0EB1064A00E00022694605F10C0014
:100D700000F094FEF3E70000080000204923000083
:100D8000952100000FB408B50399002904D004AAE6
:100D900000926A4600F00FF801B05DF814FB10B540
:100DA00082680446002A05D0D4E9040321689847E4
:100DB0000020A06010BD2DE9FC4791460C00804644
:100DC00076D014F8011B39B125290ED04046FFF723
:100DD00019FD20780028F4D198F80C00002867D07D
:100DE0004046BDE8FC47FFF7DABF0020012221782A
:100DF0002B291BD02D2902D0302908D102E040F048
:100E0000010001E040F00200641C002AEFD100253F
:100E10002A290ED02178A1F130020A2A11D205EB3D
:100E2000850201EB4205641C303DF1E740F004000F
:100E3000EAE7D9F800100B1DC9F800300968641CF6
:100E40000D44217800232E290BD114F8011FA1F1A4
:100E500030020A2A05D203EB830201EB4203303B46
:100E6000F3E76C290DD068290BD0692921D00BDC60
:100E7000252918D0582931D063290ED0642915D1DD
:100E800017E014F8011FECE7702969D0732932D0FC
:100E900075291BD0782909D120E0D9F80000011D5F
:100EA000C9F8001001784046FFF7ACFC641C90E7DD
:100EB0006CE0D9F800100A1DC9F800200968CDE9D6
:100EC00000500A224046FFF7C1FCEFE7D9F80010B6
:100ED0000A1DC9F8002009680A2206E0D9F80010A6
:100EE0000A1DC9F8002009681022CDE900504046CB
:100EF00001F0BCFADAE7D9F8001000270A1DC9F89A
:100F000000200E68C00705D112E04046761C7F1C09
:100F1000FFF778FC31780029F7D104E02021404622
:100F20006D1EFFF76FFCBD42C0D9002DF6D1BDE7A5
:100F30004EB13046FFF71AFA074604E0202140463A
:100F40006D1EFFF75FFCBD4206D9002DF6D103E010
:100F50004046761CFFF756FC31780029F8D1A5E70A
:100F6000D9F80000011DC9F800100568302140467D
:100F7000FFF748FC78214046FFF744FC0820002199
:100F8000CDE90001034610222946B0E7BDE8FC8701
:100F90002DE9FF411C46DDE90A7815460E466846F4
:100FA00000F060F846EA450141EA840141EA07227F
:100FB00042EA0841009A00EB8200C0F80017BDE841
:100FC000FF812DE9FF411C46DDE90A7815460E46F2
:100FD000684600F055F846EA450141EA840141EAD5
:100FE000072242EA0841009A00EB8200C0F800178D
:100FF000BDE8FF811CB5002100910B460122019143
:10100000FFF7C6FF1CBD1CB5002100910B46012255
:101010000191FFF7D6FF1CBD1CB500220B460092C4
:1010200011460192FFF7B4FF1CBD1CB500220B4610
:10103000009211460192FFF7C4FF1CBD1CB50021B0
:1010400000910B46012201911146FFF7A1FF1CBD43
:101050001CB5002100910B46012201911146FFF7BA
:10106000B0FF1CBD0168202902D24FF0A04070479C
:1010700001F01F01016001487047000000030050AB
:101080000168202902D24FF0A040704701F01F01F3
:1010900001600148704700000003005001B5684638
:1010A000FFF7E0FF009A01219140C0F8081508BD44
:1010B00001B56846FFF7E4FF009A01219140C0F8AE
:1010C000081508BD30B5124B01460020D3F8104476
:1010D000224609E0157A854205D1401C0A28F7DB33
:1010E0004FF0FF3030BD5268002AF3D1421CF9D0D6
:1010F0000872D3F810242AB152684A60D3F8102439
:10110000516030BD0022C3F810144A6030BD0000A9
:1011100064020020F0B595B01C4615460F460846FF
:101120001A9E00F05DFB182109A8FFF714F90E962E
:10113000CDE909540023082203A9384600F065FBD5
:1011400005980690BDF81000ADF81C00BDF812001F
:10115000ADF81E0000208DF821000398082600F04D
:101160000300012802D0022818D032E00398334649
:10117000850AC0F3C2008DF8200003980FA9C0F3C0
:101180008314A200384600F040FB09A8009006AB8B
:1011900022460FA9284600F07FFA1AE00398840D32
:1011A000C0F3C2008DF82000082C01D2254600E0D3
:1011B000082533462A460FA9384600F026FB2E4460
:1011C000641B09AB06AA29460FA800F0B7F9002C4A
:1011D000EAD1384600F00AFB15B0F0BD7047012097
:1011E00000F0F6BF084810B50178084A515C19B103
:1011F000001D00F00DFE02E00C3000F01BFDBDE80C
:101200001040002000F0E4BF300000200400002067
:1012100008B5034A00924023024AFFF77BFF08BD4E
:101220008D200000640100200A4A012902EBC00061
:1012300007D0022907D0032907D0042907D00020AE
:10124000704702207047042070470079704740794A
:1012500070470000C426000010B5FFF7C0FF04214E
:101260000348FFF72FFF02490120487210BD00001C
:10127000440000202DE9F0478CB0FFF7D3FA18B1F5
:1012800000200CB0BDE8F087784C0020C4F81804AA
:10129000BFF34F8F60680290A5684FF000082840A8
:1012A00004EB800008E021680298814201D8616067
:1012B000E6E7284004EB80000C3002A9FFF75AFB58
:1012C0000028F0D103AB029901EA050204EB820287
:1012D000491CD26843F82020401C02910228F2D316
:1012E000039800F00300022802D001284ED0A5E0A8
:1012F00003985022810D8946B2EB905F00D85021AF
:101300000E4666F39F5003900831594800F01FFACB
:10131000070078D000F064FA4346082203A9384653
:1013200000F079FA029908F1080A2940681A800049
:10133000001D864223D94D4D0C3530B1C2B204EBAD
:101340008101301A90460C3104E02946F2B20025A2
:1013500090462846C6B25346384600F05CFA0AEB7F
:1013600008032DB1324629464FEA070000F053FA30
:10137000029909F1030001EB900002903AE004EBBE
:1013800081015346324638460C31EFE70398C0F3EB
:101390008311062900D3062161F389100390C0F35D
:1013A0008310801C8100324800F0D1F9070045D03D
:1013B00000F016FA4346082203A9384600F02BFA3B
:1013C00008F1080800260FE00298434600EA0501EC
:1013D000401C04EB81010290042238460C3100F0DD
:1013E0001AFA08F10408761C0398C0F38310B0427F
:1013F000EAD847B1D4F81054D4F8180468B1384684
:1014000000F0F4F92CE019E0687A012804D12A6888
:1014100028463946126890476D68002DF4D1384649
:1014200000F0E4F90020FFF71CF9D4F8180408B91B
:10143000029860600020FFF716F911E0D4F810441C
:1014400004E021682046896888476468002CF8D148
:1014500008480221008801EB004007A100F06AF86B
:10146000FFF7E0F980F001000BE7000064020020C4
:1014700004270000C00000204261636B656E647346
:1014800020666C7573686564000000002DE9F84FF4
:101490008146DFF89C80D01C15468A4680080022D1
:1014A0006946D8F80860FFF769F9B8B3009CA01C3A
:1014B0000090D8F808103040091A8F003F1DBD4237
:1014C00008EB800002D82A46514608E03A465146C9
:1014D0000C30FEF727FF1648EA1B0AEB07010C3019
:1014E000FEF720FF4FEA1947FFF7A6F947EA004247
:1014F000601C304008EB8000344008EB8401C2607F
:10150000C8684FF6C07269F3C500904365F39F50F9
:1015100020F00300801C20F00400C86098F820042C
:1015200002E000BFFFF7A6FE0028FBD1BDE8F88F60
:101530006402002000231A4600F0C8BD2DE9F047E0
:101540000E4680461C46924608293ED894F80C90D8
:10155000002020731946104600F0D0FC0025B5424B
:1015600006D218F805201AA12046FFF70BFC03E06D
:1015700019A12046FFF706FC6D1C082DEFD317A11B
:101580002046FFF7FFFB0025B54210D218F8057082
:10159000FEF7C4FE0068C05D10F03E0F01D03A4671
:1015A00000E02E220EA12046FFF7ECFB03E00DA188
:1015B0002046FFF7E7FB6D1C082DE5D301222146ED
:1015C000504600F07DFC84F80C90BDE8F0870000E8
:1015D0002025303278000000202020007C00000010
:1015E0002563000020000000104810B5FF21816035
:1015F000002101604160C0F81814C0F8141480F88C
:1016000020140B4800F0F0F800280DD109480A49D1
:101610000A4B401AC108002003E000BF23F8200055
:10162000401C8842FAD3002010BD00006402002054
:101630000427000004270000C4260000A4000020A6
:1016400002480349401AC008704700000427000000
:10165000C426000013B56846FFF7A4FA08B10020BD
:101660001CBD0248009950F831001CBDC426000082
:1016700070B508480125D0F8104480F8205405E0E2
:10168000657221682046496888476468002CF7D154
:1016900070BD0000640200202DE9FF4781460C9DCB
:1016A00000200C462F7B287398461646294618467C
:1016B00000F024FC072E42D2DFE806F004090F16E2
:1016C0001F2A360049462846FFF75CFB37E04946AB
:1016D00028462268FFF756FB31E0D4E9002349464B
:1016E0002846FFF74FFB2AE0A0680090D4E90023CA
:1016F00049462846FFF746FB21E0D4E90201CDE93F
:101700000001D4E9002349462846FFF73BFB16E0D9
:1017100004F1080007C88DE80700D4E90023494612
:101720002846FFF72FFB0AE004F108000FC88DE8F8
:101730000F00D4E9002349462846FFF723FB002287
:101740002946404600F0BCFB2F73BDE8FF872DE91A
:10175000F041858A80462D1F4819C01CB0FBF5F06A
:10176000C6B24046FFF758FA041E19D00020207177
:1017700001206071E58000272546761EC4F80080B0
:101780000BE04046FFF748FA60B16179491C61718E
:10179000286005467F1CC0F80080B742F1D3204680
:1017A000BDE8F081204600F002F80020F8E72DE9BE
:1017B000F041457901466B1E002201E00968521C88
:1017C0009A42FBD30F680146002605E038460C68B4
:1017D000FFF741FA2146761CAE42F7D3BDE8F0810F
:1017E0000121001DFFF7FCB9FFF74ABA10B5044606
:1017F0000121001DFFF70AFA10F0FF0F04D1204667
:10180000BDE81040FFF7D3BF10BD38B501240094E8
:10181000FFF78CF938BD38B500240094FFF786F93E
:1018200038BD01680A6849688068884201D9491C46
:1018300000E00021914201D1012070470020704753
:101840008068884201D9481C7047002070472DE904
:10185000F04104464FF000080E464046FEF701FFF7
:101860002046FFF7DEFF070009D0207C38B14FF09B
:1018700004080020FEF7F7FE4046BDE8F08120682E
:10188000456841682046FFF7DBFF2168486037B1B3
:10189000206801682046FFF7D3FF21680860E268EE
:1018A000012A14D0022A16D0042A19D0082A1CD0E2
:1018B0006068314605FB0200FEF734FD204600F06B
:1018C000A8FB21688A688242D3D28860D1E7616828
:1018D00030784855F2E76168308821F81500EDE767
:1018E0006168306841F82500E8E7D6E900016268E0
:1018F00002EBC502C2E90001E0E72DE9F04107462D
:101900004FF0000415000E46204611D0FEF7A9FE48
:10191000384600F07EFBA84205D32A4631463846B9
:1019200000F044FB00E005240020FEF79CFE20466A
:10193000BDE8F08110B504460020FEF792FE204677
:1019400000F067FB04460020FEF78DFE204610BD28
:101950004058002800D00120704708B500224250AE
:101960004058009008BDD0F80403084000D0012082
:1019700070474058002800D00120704708B5002269
:1019800042504058009008BD0121B1EB507F01D179
:10199000012070470020704770B50D4600F0FAFA3C
:1019A00004000FD00020FEF75CFE207920B100205B
:1019B000FEF759FE112070BD012025602071002026
:1019C000FEF751FE002070BD10B500F0E3FA0028CC
:1019D00002D000210160017110BD000001B569460F
:1019E0000548FFF734FF0448FFF71BFF002801D02C
:1019F00000F042F808BD00001C270000124A1378CE
:101A00000BB18520704751600178C90704D00F4998
:101A10000B6843F001030B600D49D1F8003223F04D
:101A20000103C1F8003240780A49400181F80004FE
:101A300001234FF0E0205903C0F88012C0F80011D4
:101A400013700020704700002000002004D50040E3
:101A500000D000400DE000E0064908B5002204482F
:101A60000A60096800910121C0F80413016008BDF3
:101A700000D0004000D1004003490120C1F8080314
:101A8000091D08607047000000D00040014902486D
:101A900000F0C6BB14010020002000402DE9F041F9
:101AA0000546007916460F4600EB40012D4A01EB32
:101AB000C00102EB810494F82A1011B10820BDE89E
:101AC000F081294951F820102868FFF765FF08B117
:101AD0001120F4E739462846FEF7DAFD66603869DA
:101AE000206030004FF001062FD03F7F4FF48E7101
:101AF0002868FFF732FF4FF4A2712868FFF72DFF27
:101B000028681A49C0F8041328684FEA4711000BE7
:101B100040B2002806DA00F00F0000F1E02080F863
:101B2000141D03E000F1E02080F800142868000B89
:101B300040B200F01F0206FA02F14009800000F1F5
:101B4000E020C0F88012C0F8001128680421C0F815
:101B500000150020A061E06184F8290044F8140F0A
:101B6000A675ACE7140100202825000080000200C3
:101B70002DE9F047054600790B4600EB400101EBEB
:101B8000C000234901EB8004284600F043F810B15F
:101B90001120BDE8F0874FF00008C4F82080A36052
:101BA000626184F828804FF48E7647463146286873
:101BB000FFF7D3FE28684FF00109C0F808902146CE
:101BC000286800F0C9FA606800BBD5F800A00EE0F4
:101BD00094F8280008B10F2716E031465046FFF769
:101BE000B7FE0028F4D02146504600F0B5FA216A2D
:101BF00060698142F1D331462868FFF7A9FE0028C9
:101C0000F9D02868C0F80C90C4F814803846C0E7B2
:101C100014010020007900EB400101EBC0000449F1
:101C200001EB80004069002800D0012070470000CF
:101C3000140100202DE9F047044600794FF0000917
:101C400000EB400101EBC000254901EB8007206853
:101C5000C0F80095786880B120682249C0F8081360
:101C600020680121000B40B200F01F0291404009A2
:101C7000800000F1E020C0F880112068D0F80C2529
:101C8000D0F81485D0F80865D0F810554FF0FF3122
:101C9000C0F81415C0F80C152068C0F80815C0F875
:101CA0001015501C02D01046FFF7A4F9B8F1FF3F01
:101CB00002D04046FFF79EF9681C02D02846FFF785
:101CC00099F9701C02D03046FFF794F92068FFF7AD
:101CD0007BFE87F82A90C7F80490BDE8F0870000E3
:101CE00014010020840202000149024800F044BBB4
:101CF00040010020002000402DE9F0410546164635
:101D000000790F46154A00EBC00102EB810494F8FC
:101D1000201011B10820BDE8F081114951F82010C0
:101D20002868FFF739FE08B11120F4E73946284644
:101D3000FEF7E9FC6660386920601EB1397F2846ED
:101D4000FEF7D8FD28680821C0F800150020A06122
:101D5000E0610121606184F82010DCE7400100208F
:101D60002C2500002DE9F04704460E460079204955
:101D700000EBC00001EB800517463046FFF704FE7C
:101D800030B1204600F036F820B11120BDE8F087D0
:101D90001020FBE76F61AE604FF49076002731466C
:101DA0002068FFF7EBFD4FF4AC7841462068FFF761
:101DB000E5FD2068AA686969C0F84425C0F848159F
:101DC000206801218160686878B9B1464946206879
:101DD000FFF7CFFD064641462068FFF7CAFD0643E0
:101DE000F4D000B10F27002068613846CEE700002C
:101DF000400100200079054900EBC00001EB8000A4
:101E00004069002800D001207047000040010020F8
:101E10002DE9F04704460079274900EBC00001EBAB
:101E2000800720684FF00009C0F80095786880B1FD
:101E300020682249C0F8081320680121000B40B235
:101E400000F01F0291404009800000F1E020C0F83E
:101E500080112068D0F80C25D0F81485D0F80865DA
:101E6000D0F810554FF0FF31C0F80C15C0F814151C
:101E70002068C0F80815C0F81015501C02D0104694
:101E8000FFF7C1F8B8F1FF3F02D04046FFF7BBF8BB
:101E9000681C02D02846FFF7B6F8701C02D0304606
:101EA000FFF7B1F82068FFF78FFD87F82090C7F89B
:101EB0000490BDE8F08700004001002010030200FC
:101EC00010B50C46017A052908D0407A38B1084887
:101ED00008A102682046FEF755FF00E01AB106A1EE
:101EE0002046FEF74FFF2046BDE81040FEF757BFE3
:101EF0007C000020257300000D0A000038B5C3885F
:101F00000D46044633B114A0009015A216A1284630
:101F1000FEF738FF217A05291CD0607A48B1A088E5
:101F2000FFF782F9164951F8202016A12846FEF73E
:101F300029FFA0880021FFF78DFB03461049207A76
:101F4000143951F8202001B02846BDE830400EA1D8
:101F5000FEF718BF38BD00001B5B306D00000000AD
:101F60001B5B313B33316D0025734C6F677320640D
:101F7000726F70706564202825642925730D0A002E
:101F80007C000020257300003C25733E2025733A19
:101F9000200000000349884201D103487047002017
:101FA0007047000000200040180000202DE9F0419B
:101FB000044600681746884605684068854201D88F
:101FC000461B02E0A068461B761CE2686068B742C8
:101FD00005FB02010CD87A434046FEF7A3F9A1683D
:101FE000E819884200D9002021680860BDE8F08126
:101FF00002FB06F52A464046FEF794F9E268BE1B4E
:10200000724308EB05006168FEF78CF920680660F2
:10201000ECE701680A684968914201D3881A704761
:102020008068801A0844401C704770B5054688696E
:102030000C4600284FF4847128460AD0FFF78DFC27
:10204000D5F81805626AE1688854606A401C6062CD
:1020500070BDFFF782FCD5F8180570BD1FB50123D0
:102060008DF80030CDE90121D0E900126846904793
:102070001FBD1FB501238DF800308DF808100192A7
:10208000D0E90012684690471FBD000070B50D4CA6
:102090000020D2B22070201D0B4D0378EB5C1BB1E9
:1020A000001DFFF75FFE02E00C30FFF761FD08B195
:1020B000FEF7CCFA6078002802D021780029FAD007
:1020C00070BD00002C000020040000202DE9F84F16
:1020D000204D924689460646984601226946184692
:1020E000AF68FEF74BFB58B3009800210446801CF4
:1020F00009E000BF00EA07035AF8212005EB83033B
:10210000401C491CDA604145F4D34FEA164AFEF7F9
:1021100093FB4AEA0041601C384005EB80003C40DC
:1021200005EB8402C160D06866F3C50068F38910CE
:1021300069F39F2020F00300401C20F00400D060D1
:1021400095F8200402E000BFFFF794F80028FBD1C7
:10215000BDE8F88F6402002070B50C4605464FF4C8
:102160008E71FFF7FAFB216AA068415C206A401C6F
:102170002062C5F81C1570BD1FB500228DF8002027
:102180000291816801914261D0E90012684690474E
:102190001FBD00001FB50A4601788DF80010416888
:1021A0000191017A8DF80810C0680390044850F836
:1021B0002210083850F82220684690471FBD0000C2
:1021C0001000002001490120087070472C000020F9
:1021D00010B588B0044620220E496846FEF7A2F8E2
:1021E00006200090C01F0190029003904FF0EB700A
:1021F00006900CB1084A00E0002269460748FEF745
:102200008DFD08B1FEF722FA0448001F447008B0A3
:1022100010BD00004C250000C5210000300000204A
:102220002DE9FF470C4605464FF40071FFF79BFB75
:1022300001274FF40178002618B34FF492794946EC
:102240002846FFF785FBE0B149462846FFF785FBA6
:10225000C5F8088394F8290000B96F6002208DF852
:102260000000D5F88004C5F880040390A0690290AE
:10227000E0680190A661E661D4E9001268469047E3
:1022800028E004212846FFF76EFB18B34FF4847151
:102290002846FFF75DFBE8B121462846FFF7C5FE5B
:1022A000616AA069884215D1E06938B1E268616A63
:1022B000A0612069E6616662E06008E094F82900A8
:1022C00000B96F60C5F80883A661E268616A2046BC
:1022D000FFF7C4FE4FF48E7841462846FFF738FBDF
:1022E00078B1206A6169884202D294F8280020B34C
:1022F00041462846FFF731FB616911B12046FFF7DF
:102300003BFF4FF4A27841462846FFF721FB002807
:1023100018D041462846FFF720FB94F8290000B169
:102320002F60A06900280DD0A661E268616A04B040
:102330002046BDE8F047FFF791BE21462846FFF74B
:102340000BFFDEE7BDE8FF871FB50A4601788DF871
:10235000001041680191017A8DF80810C06803905F
:10236000044850F82210083850F822206846904758
:102370001FBD0000100000202DE9FF410C464FF466
:10238000927705463946FFF7F4FA0026C0B1394680
:102390002846FFF7F3FA02208DF80000D5F88004F4
:1023A000C5F880040390D5F83C058DF80800E06876
:1023B0000190A661E661D4E900126846904723E0E7
:1023C0004FF4887739462846FFF7D3FAE0B139460B
:1023D0002846FFF7D3FAD5F83C15A069884213D1F7
:1023E000E06960B1E268D5F8000220F02000C5F88D
:1023F0000002E069A0612069E661E06001E0A66199
:10240000E2682046FFF735FE4FF4A27739462846AA
:10241000FFF7AFFA60B139462846FFF7AFFAA06977
:1024200030B1A661D5F83C152046E268FFF721FEE1
:102430004FF4907739462846FFF79BFA002813D0CF
:1024400039462846FFF79AFA606900280CD0D5F87B
:102450004C058DF800608DF80800A0680190666159
:10246000D4E9001268469047BDE8FF812DE9F05F8E
:102470008346DDE90A4A994690460D4608460127FB
:1024800003E000BFB0FBF8F07F1C4045FAD2B9452D
:1024900000D94F465FEACA7012D18CB15FEA8A70E8
:1024A00002D5B9F1000F01D0202607E0302605E063
:1024B00031465846641EFEF7A5F90CB1A742F7D382
:1024C0005FF00106B9F1010F02D9A9F1010903E09A
:1024D000B5FBF6F0404502D306FB08F6F2E7DFF85D
:1024E0003C9000BFB5FBF6F000FB165519F8001044
:1024F0005846FEF787F9B6FBF8F6002EF2D15FEAF0
:10250000CA7009D0002C07D0A74205D22021584616
:10251000641EFEF777F9F5E7BDE8F09F302500006F
:102520000338FDD8704701078D1A0000E91C000030
:1025300030313233343536373839414243444546F9
:1025400011120000E5110000DD110000FFFFFFFF88
:10255000FFFFFFFFFFFFFFFFFFFFFFFF0000000087
:10256000000000000000D6010701000000404040CC
:102570004040404040404141414141404040404056
:102580004040404040404040404040404005020202
:1025900002020202020202020202020202202020C1
:1025A000202020202020200202020202020290901D
:1025B000909090901010101010101010101010101B
:1025C000101010101010101002020202020288886F
:1025D000888888880808080808080808080808087B
:1025E0000808080808080808020202024000000063
:1025F0006D2500007761726E696E670064656275B3
:10260000670000001B5B313B33306D001B5B306D9E
:10261000000000001B5B313B33316D001B5B313B25
:1026200033326D001B5B313B33336D001B5B313B41
:1026300033346D001B5B313B33356D001B5B313B2D
:1026400033366D001B5B313B33376D00696E666F4F
:10265000000000006572726F72000000726E670009
:1026600071756575652E6D5F72616E645F706F6FF9
:102670006C00000050525300524E470055415254D6
:1026800000000000554152544500000062616C6C2E
:102690006F632E6C6F675F6D656D706F6F6C0000A0
:1026A000617070003427000000000020C4000000AA
:1026B000B0050000F8270000C4000020C425000079
:1026C000C00500005C26000000000000602600003D
:1026D00000000003742600000000000078260000BF
:1026E000000000007C26000000000000842600009E
:1026F000000000008C26000000000003A02600005F
:102700000000030358000020500000205800002063
:10271000A4010020BC0000201800000008010020D7
:10272000C400002040000000010000000000000084
:10273000A8000020000000000000000000000000D1
:102740000000000000000000000000000000000089
:102750000000000000000000000000000000000079
:102760000000000000000000002000400000000009
:102770000020004000000000402500000000000094
:102780000000000000000000000000000000000049
:102790000000000000000000000000000000000039
:1027A00054260000F42500004C260000FC25000003
:1027B0000C26000004260000142600001C26000041
:1027C000242600002C260000342600003C260000B1
:1027D000442600000090D00300000000000000002C
:1027E00000000000000000000000000000000000E9
:0827F0000000000000000000E1
:0400000500000201F4
:00000001FF
